:1000000012C02BC02AC029C028C027C026C025C0C6
:1000100024C087C122C058C120C01FC01EC01DC03F
:100020001CC01BC01AC011241FBECFE5D4E0DEBF28
:10003000CDBF10E0A0E6B0E0EAEBF3E002C005902F
:100040000D92A036B107D9F710E0A0E6B0E001C0EC
:100050001D92A636B107E1F769C0D2CF20E030E0AB
:100060002817390748F440E0475E483CE8F32F5F23
:100070003F4F28173907B8F308958EB58C7F8460F9
:100080008EBD8FB58C7F8FBD8EB5877F80618EBD15
:100090008FB58F7B80688FBD8FB58F7E80628FBD5F
:1000A0008FEF90E097BD86BD1BBC1ABC19BC18BC75
:1000B000089580B7846080BF87B38F6387BB88B3A0
:1000C000817E816288BB84B3837C836084BB85B37B
:1000D000807C85BB81B384EF81BB82B380E282BB2D
:1000E0008FB581EA8FBD8EB5827282608EBD86B17A
:1000F00086E886B98FB780688FBF08958BB11BB82B
:100100008AB11AB880B580E880BD80B5807780BD9F
:1001100089B187E689B9089583B78C7F846083BFEE
:1001200089B78E7F89BF88EC82BF0895CFE5D4E080
:10013000DEBFCDBFBEDFA1DF9698E0DFEDDF10921E
:10014000600010926500579A549A8091650080FF74
:10015000FCCF809165008E7F809365008091610067
:1001600090916200A0916300B09164008F739070D1
:10017000A070B07080319105A105B10509F446C0A9
:1001800081319105A105B1055CF40097A105B10588
:1001900009F491C00C97A105B10509F48CC091C078
:1001A00080329105A105B10581F081329105A1054B
:1001B000B10534F44197A105B10509F449C081C0E6
:1001C0008197A105B10579F07CC0A99AA89A1BBCBA
:1001D0001ABC19BC18BC82B38F7E806282BB88B304
:1001E0008F7E80620DC0A998A8981BBC1ABC19BC50
:1001F00018BC82B38F7D806182BB88B38F7D8061A4
:1002000088BB80EC90E09BBD8ABD13C0A99AA898DA
:10021000C8B5D9B5209781F019BC18BC80E593EC1E
:100220001DDF80E593EC1ADF80E593EC17DF80ECAF
:1002300090E099BD88BD45C0DBBDCABDD9BDC8BD74
:1002400082B38F7E806282BB88B38F7D806121C044
:10025000CAB5DBB5209781F01BBC1ABC80E593ECD6
:10026000FDDE80E593ECFADE80E593ECF7DE80ECD2
:1002700090E09BBD8ABD25C0A89AA998DBBDCABDE8
:10028000D9BDC8BD82B38F7D806182BB88B38F7EAC
:10029000806288BB80EC90E09BBD8ABD99BD88BD23
:1002A00080E593ECDBDE80E593ECD8DEDBBDCABDF8
:1002B000D9BDC8BD06C0A998A8981BBC1ABC19BC5A
:1002C00018BC1092600040CF1F920F920FB60F9291
:1002D00011248F939F93AF93BF93549880B78160FD
:1002E00080BF84EE82BF88B7816088BF89B7816094
:1002F00089BF81E090E0A0E0B0E08093610090933E
:100300006200A0936300B093640081E0809360007A
:10031000BF91AF919F918F910F900FBE0F901F9043
:1003200018951F920F920FB60F9211248F939F93DF
:10033000AF93BF9389EC82BF80916100909162007E
:10034000A0916300B0916400880F991FAA1FBB1F82
:100350008093610090936200A0936300B093640067
:10036000809911C08091610090916200A09163001A
:10037000B091640081608093610090936200A093CB
:100380006300B0936400809160008F5F8093600091
:10039000809160008E3041F489B78E7F89BF809153
:1003A0006500816080936500BF91AF919F918F91AF
:0A03B0000F900FBE0F901F901895DC
:00000001FF
